:03000000020800F3
:0C080000787FE4F6D8FD758140020847BF
:10092B00415445300D0A000000000000000000009B
:10093B000000000000000000000000000000415417
:10094B002B43495053544152543D22544350222C73
:10095B00223139322E3136382E322E313038222C8C
:07096B00383038300D0A009E
:10099E00C100C1021E230000000000000000000084
:1009AE000000000000000000000000000000000039
:0709BE00000000000122000F
:070A3B0053A27F43A28022B9
:040A420053A27F221A
:0E0A160000007F7F7EE97D94DDFEDEFCDFFACE
:010A240022AF
:080A32007F0B7EF6DEFEDFFC07
:010A3A002299
:1009C60053877F759850438E40538EFE53890F434D
:0D09D6008920758BFD758DFDC2ABD28E2280
:1009E300200003300213120A427B007A007923129B
:0A09F3000972C200C202120A3B2280
:10088C00C203C204120A16120A16120A161209C65A
:10089C00E4F59175923FD2ACD2AFD29C120A3B12C6
:1008AC000A32120A3220030ED2037BFF7A09792B0B
:1008BC00120972120A161209E330031120040ED227
:1008CC00047BFF7A097949120972120A161209E39C
:0208DC0080D3C7
:030023000208DEF2
:0908DE00C0E0C0D075D000C000DC
:1008E700309833C298E521B40D10E599B40A0BE5A9
:1008F7002264016005D200752200C2987423252264
:10090700F8A6998599210522D3E5226480949D4014
:0D09170005752200D202309904C299C20178
:07092400D000D0D0D0E0327A
:0D0A250030010122EFD201F5992001FD22E0
:100972008B088A09890AAB08AA09A90A1209FD602B
:100982001A120A32AB08050AE50AAA097002050919
:0C09920014F91209FDFF120A2580DB2277
:10080C0002088CE493A3F8E493A34003F68001F26E
:10081C0008DFF48029E493A3F85407240CC8C333ED
:10082C00C4540F4420C8834004F456800146F6DFBC
:10083C00E4800B010204081020408090099EE47EA5
:10084C00019360BCA3FF543F30E509541FFEE493B1
:10085C00A360010ECF54C025E060A840B8E493A378
:10086C00FAE493A3F8E493A3C8C582C8CAC583CAA3
:10087C00F0A3C8C582C8CAC583CADFE9DEE780BE5B
:0109C5000031
:1009FD00BB010689828A83E0225002E722BBFE02F8
:090A0D00E32289828A83E493222A
:00000001FF
